:100000000C945A000C9477000C9477000C947700B1
:100010000C9477000C9477000C9477000C94770084
:100020000C9477000C9477000C9477000C94770074
:100030000C9477000C9477000C9477000C94770064
:100040000C948A010C9477000C9477000C94770040
:100050000C9477000C9477000C9477000C94770044
:100060000C9477000C947700000024272A000025C8
:10007000282B000023262904040404040404040299
:100080000202020202030303030303010204081035
:100090002040800102040810200102040810200002
:1000A0000000070002010000030406000000000039
:1000B0000000000011241FBECFEFD4E0DEBFCDBF93
:1000C00011E0A0E0B1E0ECE3F6E002C005900D9293
:1000D000A030B107D9F711E0A0E0B1E001C01D9256
:1000E000A830B107E1F70E9483010C941C030C9423
:1000F00000000F931F93182F062F60E082E10E94EB
:10010000850261E08DE00E94850261E070E080E0A0
:1001100090E00E94F5011BB961E081E10E94850237
:1001200061E070E080E090E00E94F50160E081E134
:100130000E948502013011F461E001C060E089E0B5
:100140000E94850260E08AE00E94850261E070E022
:1001500080E090E00E94F50161E08AE00E94850263
:1001600064E670E080E090E00E94F5011F910F913D
:1001700008951F93182F61E082E10E94850260E0DC
:100180008DE00E94850260E089E00E9485021BB933
:1001900061E081E10E94850261E070E080E090E032
:1001A0000E94F50160E081E10E9485021F9108959F
:1001B0008FE00E94D0020197D9F360E083E10E94B2
:1001C000850260E082E10E94850260E08DE00E948D
:1001D000850260E089E00E94850260E080E10E9483
:1001E000850261E088E00E94850261E08AE00E9469
:1001F000850261E08BE00E94850261E070E080E0B2
:1002000090E00E94F50160E08EE00E94850261E0CE
:1002100070E080E090E00E94F50180E40E94B90067
:1002200061E089E90E94790080E40E94B90060E001
:1002300081EC0E94790068EE73E080E090E00E941B
:10024000F50161E08EE00E9485021BB860E08BE062
:100250000E94850260E08AE00E94850260E083E1FE
:100260000E94850260E082E10E94850260E08DE0EC
:100270000E94850260E089E00E94850260E080E1E2
:100280000E94850260E088E00E94850208951BB804
:100290008FEF8AB961E088E00E94670260E08CE03D
:1002A0000E94670261E08BE00E94670261E08AE0E1
:1002B0000E94670261E089E00E94670261E08DE0D0
:1002C0000E94670261E082E10E94670261E083E1CF
:1002D0000E94670261E08EE00E94670261E080E1B7
:1002E0000E94670261E081E10E94670260E08FE0A6
:1002F0000E94670261E08FE00E94850261E08EE06B
:100300000E94850208950E942D020E9447010E94CA
:10031000D800FDCF1F920F920FB60F9211242F938A
:100320008F939F93AF93BF938091000190910101B0
:10033000A0910201B09103018050904CAF4FBF4F8C
:100340008093000190930101A0930201B0930301F7
:1003500027C08091000190910101A0910201B0910C
:10036000030180589E43A040B040809300019093C9
:100370000101A0930201B0930301809104019091C7
:100380000501A0910601B09107010196A11DB11DC3
:100390008093040190930501A0930601B093070197
:1003A0008091000190910101A0910201B09103019F
:1003B00081589E43A040B04060F6BF91AF919F919D
:1003C0008F912F910F900FBE0F901F9018958FB7A0
:1003D000F89420910401309105014091060150915B
:1003E00007018FBFB901CA010895EF92FF920F93E1
:1003F0001F937B018C018FB7F894409104015091B9
:10040000050160910601709107018FBF2FB7F89425
:100410008091040190910501A0910601B09107011E
:100420002FBF841B950BA60BB70B8E159F05A0073E
:10043000B10760F31F910F91FF90EF90089501971E
:1004400059F0FC01EE0FFF1FEE0FFF1F32978FB721
:10045000F8943197F1F78FBF0895789484B582604E
:1004600084BD84B5816084BD85B5826085BD85B558
:10047000816085BDEEE6F0E0808181608083E1E807
:10048000F0E0808182608083808181608083E0E809
:10049000F0E0808181608083E1EBF0E08081846026
:1004A0008083E0EBF0E0808181608083EAE7F0E028
:1004B000808184608083808182608083808181608C
:1004C00080838081806880831092C1000895282FE6
:1004D00030E0C90185579F4FFC01949129583F4F47
:1004E000F9018491882381F0E82FF0E0E859FF4F6B
:1004F000E491F0E0662329F480819095892380833C
:1005000008958081892B80830895482F50E0CA0187
:1005100081569F4FFC012491CA0185579F4FFC01D2
:10052000949149585F4FFA0134913323C1F122234A
:1005300031F1233021F4809180008F7705C0243081
:1005400031F4809180008F7D8093800018C021302D
:1005500019F484B58F7704C0223021F484B58F7DDF
:1005600084BD0DC0263021F48091B0008F7705C086
:10057000273029F48091B0008F7D8093B000E32F65
:10058000F0E0E359FF4FE491F0E0662329F4808125
:1005900090958923808308958081892B8083089595
:1005A000482F50E0CA0181569F4FFC012491CA0197
:1005B00085579F4FFC01949149585F4FFA01349140
:1005C000332319F420E030E035C0222331F1233009
:1005D00021F4809180008F7705C0243031F4809120
:1005E00080008F7D8093800018C0213019F484B57D
:1005F0008F7704C0223021F484B58F7D84BD0DC077
:10060000263021F48091B0008F7705C0273029F47F
:100610008091B0008F7D8093B000E32FF0E0EE5822
:10062000FF4FE491F0E0808120E030E0892311F079
:0C06300021E030E0C9010895F894FFCFEC
:00000001FF
